:020000040800F2
:10000000A807002031020008FB210008F3210008A6
:10001000F7210008ED070008F92A00080000000099
:10002000000000000000000000000000D9230008CC
:10003000F107000800000000FD210008DB23000894
:100040005502000855020008550200085502000834
:100050005502000855020008550200085502000824
:100060005502000855020008550200085502000814
:100070005502000855020008550200085502000804
:1000800055020008550200085502000855020008F4
:1000900055020008550200085502000855020008E4
:1000A00055020008550200085502000855020008D4
:1000B00055020008550200085502000855020008C4
:1000C00055020008550200085502000855020008B4
:1000D00055020008A92A0008550200085502000828
:1000E000F5070008550200085502000855020008EF
:1000F0005502000855020008550200085502000884
:100100005502000855020008550200085502000873
:100110005502000855020008550200085502000863
:100120005502000855020008550200085502000853
:100130005502000855020008550200085502000843
:100140005502000855020008550200085502000833
:100150005502000855020008550200085502000823
:100160005502000855020008550200085502000813
:100170005502000855020008550200080000000062
:10018000550200085502000800F002F800F041F89E
:100190000AA090E8000C82448344AAF10107DA45E2
:1001A00001D100F036F8AFF2090EBAE80F0013F0F3
:1001B000010F18BFFB1A43F0010318477C2C000005
:1001C0009C2C0000103A24BF78C878C1FAD8520796
:1001D00024BF30C830C144BF04680C6070470000C1
:1001E0000023002400250026103A28BF78C1FBD840
:1001F000520728BF30C148BF0B607047642900F028
:10020000F580002070471FB502F004FE1FBD10B539
:1002100010BD00F0D9F91146FFF7F5FF02F00EFD11
:1002200000F0F7F903B4FFF7F2FF03BC02F082FC21
:100230000C48016841F4700101600B4880470B488D
:100240000047FEE7FEE7FEE7FEE7FEE7FEE7FEE724
:10025000FEE7FEE7FEE7000005480649044A064BB4
:100260007047000088ED00E0E523000889010008E0
:10027000A8030020A8070020A8030020704753EA25
:10028000020C00F069802DE9F04B4FF00006002BC6
:100290001FBFB3FA83F503FA05F424FA05F65E40AE
:1002A00012BF1643B2FA82F502FA05F4C5F1200531
:1002B0001EBF22FA05FC44EA0C04203556EA044C21
:1002C0004FEA144418BF641C4FF000084FF00009B7
:1002D000904271EB030C39D3002919BFB1FA81F7B1
:1002E00001FA07F6B0FA80F700FA07F6C7F120071F
:1002F0001EBF20FA07FC46EA0C062037B6FBF4FCCA
:10030000A7EB0507103F07F01F0BCBF120060CFAF7
:100310000BFB2CFA06F644BFB3460026202FA4BFE1
:100320005E464FF0000B5BEA060C08BF4FF0010B76
:1003300019EB0B09ABFB027C48EB0608C01B06FB64
:1003400002CC0BFB03CC71EB0C01C1E70B46024660
:1003500041464846BDE8F08B13B54FF000004FF022
:100360000001AFF30080BDE81C4070470FB40449A2
:1003700010B503AA029800F0F9F810BC5DF814FB60
:10038000080000202DE9F0410E46044600202062BE
:100390002046E168884730B3252805D0D4E90121FB
:1003A0009047206A401CF2E7E16820460027884712
:1003B000050018D0A5F14100192802D820354FF4C6
:1003C00000673246294620462760FFF717FF40B1F5
:1003D000012804D0F61D26F007060836D8E7361D9A
:1003E000D6E72846DAE7206ABDE8F0812DE9F0413A
:1003F0000646002410687529314616A510D0AFF3C3
:100400000080002802DA404213A507E031688A071D
:1004100001D512A502E0490704D511A5012401E088
:10042000AFF3008000210A2206F1240709E0B0FBA7
:10043000F2FCB0FBF2F302FB1C003030785418469B
:10044000491C0028F3D123462A463046BDE8F04136
:1004500000F033B8000000002D0000002B00000069
:10046000200000004FF0000200B513469446964667
:10047000203922BFA0E80C50A0E80C50B1F12001B7
:10048000BFF4F7AF090728BFA0E80C5048BF0CC065
:100490005DF804EB890028BF40F8042B08BF7047C3
:1004A00048BF20F8022B11F0804F18BF00F8012B35
:1004B000704770477047704770472DE9F0470D4609
:1004C00099469246044600F124080168880604D53E
:1004D000E06921F01001216000E00120A84201DD67
:1004E000471B00E00027A1697A1902EB0900081AEE
:1004F000A0612078C00602D42046AFF30080002619
:1005000008E0D4E901211AF806009047206A401C4F
:10051000761C20624E45F4DB2078C0060AD52046C2
:10052000AFF3008006E0D4E9012130209047206A33
:10053000401C2062381EA7F10107F4DC07E0D4E973
:10054000012118F805009047206A401C2062281EEF
:10055000A5F10105F3DC2046AFF30080207800060A
:1005600002D50220BDE8F0870120FBE7074B70B5FC
:100570000D467B4400F011F80446284600F020F8B0
:1005800010B14FF0FF3070BD204670BD57260000FF
:1005900001694A1C02610878704700B58FB0CDE947
:1005A00001310021059105497944CDE90310114637
:1005B0006846FFF7E7FE0FB000BD0000E5FFFFFF54
:1005C000007B00F080007047754600F02BF8AE46C7
:1005D00005006946534620F00700854618B020B54F
:1005E000FFF73AFEBDE820404FF000064FF000074D
:1005F0004FF000084FF0000B21F00701AC46ACE8CB
:10060000C009ACE8C009ACE8C009ACE8C0098D4637
:10061000704710B50446AFF300802046BDE8104097
:10062000FFF700BE004870474403002000B587B0C4
:1006300000BF00BF002001903248006840F0400039
:10064000304908600846006800F04000019000BF93
:1006500000BF00BF00BF00BF002001900846006837
:1006600040F0400008600846006800F0400001903B
:1006700000BF00BF00BF00BF00BF002001900846C0
:10068000006840F0400008600846006800F0400044
:10069000019000BF00BF00BFC81402901A48039029
:1006A0000120049002A9194800F028F90122002134
:1006B000282000F092FA282000F07FFA4FF48040C2
:1006C00002900120039004900220059002A90F4897
:1006D00000F014F9012291030C4800F011FA4FF4D4
:1006E000004002900120039004900220059002A98E
:1006F000064800F003F90122D103044800F000FA93
:1007000007B000BD30380240000021100018024040
:1007100010B586B04FF47A73182269461E4800F06F
:100720000DFF9DF815101D4A1D48006811549DF8D5
:1007300016101B480068401C11549DF817101848EB
:100740000068801C115416480068C01C14490860D9
:1007500008460068F0281DDB00224FF400411148D4
:1007600000F0CEF910A0FFF701FE002405E00B48D1
:10077000015D10A0FFF7FAFD641CF02CF7DB0FA061
:10078000FFF7F4FD0122D103064800F0B9F900207B
:100790000349086006B010BD5C0200203001002053
:1007A0001C000020001802400D0ABFAACABC0D0A96
:1007B0000000000025640D0A000000000D0ABDE1E4
:1007C000CAF80D0A0000000010B500224FF40041E5
:1007D000054800F095F9012002F0B8F90122D10393
:1007E000014800F08DF910BD0018024000BFFEE77F
:1007F0007047000010B50A48006800F4006070B14E
:100800004FF40060064908600648007828B9FFF7F1
:10081000DBFF01200349087001E0FFF779FF10BDFD
:10082000143C01402000002070B50446A56D00F086
:1008300073F9064694F83500022808D080206065D8
:1008400000BF002084F8340000BF012070BD206884
:10085000006820F01600216808602068406920F0D8
:10086000800021684861206C08B9A06C28B120681C
:10087000006820F00800216808602068006820F007
:100880000100216808600FE000F046F9801B052890
:100890000AD92020606500BF002084F8340000BF22
:1008A000032084F83500D1E72068006800F00100DB
:1008B0000028E9D194F85C103F208840A86000BF70
:1008C000002084F8340000BF012084F835000020A7
:1008D000BCE7014691F83500022803D08020486526
:1008E00001207047052081F835000868006820F075
:1008F00001000A6810600020F3E70000F8B5024626
:100900000B460025002400200021DEE0012606FA27
:1009100001F51E6806EA0504AC4275D11E7906F0A1
:100920000306012E04D01E7906F00306022E13D111
:1009300090684F000326BE40B0434F00DE68BE40C3
:1009400030439060506801268E40B0431E79C6F354
:1009500000168E40304350601E7906F00306032EC9
:1009600009D0D0684F000326BE40B0434F009E68B8
:10097000BE403043D0601E7906F00306022E13D12C
:10098000CF0802F1200656F827004E07F70E0F2673
:10099000BE40B0434F07FF0E1E69BE403043CF0834
:1009A00002F1200646F8270010684F000326BE40DB
:1009B000B0431E7906F003064F00BE40304310607E
:1009C0005E6806F08056B6F1805F7DD100BF0026DC
:1009D0000096404E366846F480463E4F3E603E46A6
:1009E000366806F48046009600BF00BF3A4E8F0876
:1009F00056F827008E07370F0F26BE40B043374EFC
:100A0000B24202D1002624E05EE0354EB24201D16E
:100A100001261EE0334EB24201D1022619E0324EC9
:100A2000B24201D1032614E0304EB24201D1042675
:100A30000FE02F4EB24201D105260AE02D4EB24200
:100A400001D1062605E02C4EB24201D1072600E076
:100A500008268F073F0FBE4030431F4E8F0846F8D1
:100A60002700264E3068A0435E6806F48036B6F54F
:100A7000803F00D12043214E3060361D3068A043B6
:100A80005E6806F40036B6F5003F00D120431B4EE9
:100A9000361D3060361D3068A0435E6806F480164F
:100AA000B6F5801F00D12043144E08363060361D45
:100AB0003068A0435E6806F40016B6F5001F00D14A
:100AC00020430E4E0C363060491C1029FFF41EAF37
:100AD000F8BD0000443802400838014000000240E0
:100AE0000004024000080240000C024000100240D6
:100AF0000014024000180240001C0240003C01406B
:100B00000AB1816101E00B0483617047014800680C
:100B1000000C7047002004E00148006870470000A6
:100B2000100000200348006803490978084401497F
:100B300008607047100000201800002010B50A4817
:100B4000006840F40070084908600846006840F4F6
:100B500080600860032000F07FF80F2000F006F8A6
:100B600000F02AF8002010BD003C024070B5044699
:100B70000E4800784FF47A71B1FBF0F00C49096827
:100B8000B1FBF0F5284600F067FF08B1012070BD09
:100B9000102C07D200222146501E00F01EF80548F6
:100BA000046001E00120F2E70020F0E718000020D7
:100BB000000000201400002070470146084600286D
:100BC00009DB00F01F0301229A4043099B0003F157
:100BD000E023C3F8002100BF70472DE9F05F804695
:100BE0000D461646002701F089FF074639462A467A
:100BF000334601F00700C0F1070ABAF1040F02D929
:100C00004FF0040A01E0C0F1070AD14600F1040ADE
:100C1000BAF1070F02D24FF0000A01E0A0F1030A77
:100C2000D4464FF0010A0AFA09FAAAF1010A0AEABF
:100C3000020A0AFA0CFA4FF0010B0BFA0CFBABF1AB
:100C4000010B0BEA030B4AEA0B042146404601F074
:100C50005DFFBDE8F09F000000BF00F00702064BFB
:100C600019684FF6FF031940044B0B4343EA022176
:100C7000014B196000BF70470CED00E00000FA0561
:100C800070B504460D460CB9012070BD5848006887
:100C900000F00700A84209D255490D7008460068C7
:100CA00000F00700A84201D00120EEE7207800F014
:100CB000020002281DD1207800F00400042805D18C
:100CC0004C48006840F4E0504A490860207800F041
:100CD0000800082805D14748006840F460404549AD
:100CE00008604448006820F0F000A16808434149CA
:100CF0000860207800F00100A8B36068012807D1DF
:100D00003C4808380068C0F34040B8B90120BCE74F
:100D10006068022802D06068032807D13548083887
:100D20000068C0F3406048B90120AEE73148083898
:100D30000068C0F3400008B90120A6E72D4800680C
:100D400020F00300616808432A490860FFF7E4FEC9
:100D5000064609E0FFF7E0FE801B41F28831884239
:100D600002D9032091E707E02248006800F00C0058
:100D70006168B0EB810FEDD11D48006800F00700FD
:100D8000A84209D91A490D700846006800F007000A
:100D9000A84201D0012078E7207800F00400042860
:100DA00007D11448006820F4E050E1680843114975
:100DB0000860207800F00800082808D10D48006875
:100DC00020F46040216940EAC1000A49086000F04F
:100DD0003FF808490968C1F30311074A515CC8404C
:100DE0000649086006480068FFF7C0FE00204CE78F
:100DF000003C0240083802401E2E0008000000207F
:100E00001400002001480068704700000000002026
:100E100000B5FFF7F7FF04490968C1F38221034ACF
:100E2000515CC84000BD0000083802402E2E00086A
:100E300000B5FFF7E7FF04490968C1F34231034AEF
:100E4000515CC84000BD0000083802402E2E00084A
:100E50002DE9F047002400250026A146254800681A
:100E600000F00C0020B1042805D008283AD105E094
:100E7000DFF8849039E0DFF8849036E01D48001FE9
:100E8000006800F03F041B48001F006800F4800069
:100E900078B11A481749091F0968C1F38811A0FBE6
:100EA00001700146224600233846FFF7E8F905465F
:100EB0000EE011480F49091F0968C1F38811A0FB12
:100EC00001700146224600233846FFF7D8F905464F
:100ED0000848001F0068C0F30140401C4600B5FBF5
:100EE000F6F902E0DFF8109000BF00BF4846BDE809
:100EF000F0870000083802400024F40000127A0055
:100F0000F8B504460CB90120F8BD207800F00100C6
:100F1000002874D0F948006800F00C0004280DD0B7
:100F2000F648006800F00C00082813D1F348001FB1
:100F3000006800F48000B0F5800F0BD1EF4808384E
:100F40000068C0F34040002859D06068002856D19E
:100F50000120D9E700BF6068B0F5803F08D1E748BD
:100F60000838006840F48030E449083908601EE021
:100F70006068B0F5A02F0DD1E0480838006840F453
:100F80008020DE49083908600846006840F4803057
:100F900008600CE0D9480838006820F48030D74950
:100FA000083908600846006820F48020086000BF07
:100FB000606890B1FFF7B0FD054606E0FFF7ACFDB5
:100FC000401B642801D903209EE7CC4808380068FC
:100FD000C0F340400028F1D011E0FFF79DFD054629
:100FE00006E0FFF799FD401B642801D903208BE739
:100FF000C24808380068C0F340400028F1D120788A
:1010000000F0020002285FD1BC48006800F00C002C
:1010100058B1BA48006800F00C0008281CD1B74845
:10102000001F006800F48000B0B9B44808380068B8
:10103000C0F3400020B1E068012801D0012063E73F
:10104000AE480838006820F0F800216940EAC10085
:10105000AA490839086037E0E06800B30120A849D0
:101060000860FFF759FD054606E0FFF755FD401BF8
:10107000022801D9032047E7A04808380068C0F3D8
:1010800040000028F1D09D480838006820F0F800A2
:10109000216940EAC10099490839086014E000203C
:1010A00097490860FFF738FD054606E0FFF734FD75
:1010B000401B022801D9032026E790480838006821
:1010C000C0F340000028F1D1207800F00800082883
:1010D0002CD16069A8B101208A490860FFF71CFD86
:1010E000054606E0FFF718FD401B022801D9032042
:1010F0000AE782486C300068C0F340000028F1D055
:1011000014E000207F490860FFF706FD054606E071
:10111000FFF702FD401B022801D90320F4E67748BF
:101120006C300068C0F340000028F1D1207800F056
:101130000400042870D1002770483830006800F09F
:10114000805090B900BF002000906C483830006893
:1011500040F080506949383108600846006800F066
:101160008050009000BF00BF01276748006800F46E
:101170008070B0B96448006840F4807062490860CB
:10118000FFF7CAFC054606E0FFF7C6FC401B022835
:1011900001D90320B8E65C48006800F4807000289C
:1011A000F2D000BFA068012808D154486830006818
:1011B00040F001005149683108601DE0A068052831
:1011C0000DD14E486830006840F004004B4968314A
:1011D00008600846006840F0010008600CE04748DD
:1011E0006830006820F00100444968310860084612
:1011F000006820F00400086000BFA068A8B1FFF7F5
:101200008BFC054609E0FFF787FC401B41F2883163
:10121000884202D9032077E626E038486830006823
:10122000C0F340000028EED013E0FFF775FC054640
:1012300008E0FFF771FC401B41F28831884201D978
:10124000032061E62D4868300068C0F340000028A4
:10125000EFD1012F07D129483830006820F08050A5
:1012600026493831086000BFA069002845D02348CE
:10127000006800F00C0008285DD0A069022845D164
:1012800000201F490866FFF747FC054606E0FFF708
:1012900043FC401B022801D9032035E617480838D3
:1012A0000068C0F340600028F1D1D4E90701084389
:1012B000616A40EA81110122A06AC2EB500041EA52
:1012C00000412C20005D41EA00600C49091F0860C4
:1012D00001200B490866FFF71FFC054606E0FFF7F3
:1012E0001BFC401B022801D903200DE603480838E7
:1012F0000068C0F340600028F1D049E0083802409F
:1013000000004742800E4742007000400020214903
:101310000866FFF701FC054606E0FFF7FDFB401BF2
:10132000022801D90320EFE51B480068C0F34060A4
:101330000028F2D12CE0A069012800D1E4E516488C
:10134000001D0668A069012820D006F48001E0692C
:1013500081421BD106F03F01206A814216D147F637
:10136000C0703040616AB0EB811F0FD106F440318C
:101370000122A06AC2EB5000B1EB004F06D106F08B
:1013800070612C20005DB1EB006F01D00120BBE546
:101390000020B9E5000047420038024010B504467D
:1013A0000CB9012010BD606A38B96068B0F5827F61
:1013B00000D105E00021E16102E0002121616161CD
:1013C000A06AB0F5005F00D100BF94F8510028B9C1
:1013D000002084F85000204600F050F8022084F8E5
:1013E00051002068006820F0400021680860A08853
:1013F00000F48270218901F404410843A18901F4B9
:1014000000610843217C01F002010843217D01F0C5
:1014100001010843218B01F400710843217F01F091
:10142000380108432021095D01F080010843218D26
:1014300001F400510843216808600421A06901EA11
:10144000104094F8241001F010010843216848600E
:10145000A06AB0F5005F03D1A08D80B22168086159
:101460002068C06920F400602168C86100206065C0
:10147000012084F85100002094E7000010B586B0E8
:1014800004462A49206888424DD100BF00BF002091
:1014900000902748006840F002002549086008468F
:1014A000006800F00200009000BF00BF00BF00BF56
:1014B00000BF002000900846006840F0020008606D
:1014C0000846006800F00200009000BF00BF00BFA7
:1014D00000BF00BF002000900846006840F00100F7
:1014E00008600846006800F00100009000BF00BFDF
:1014F00000BF0820019002200290012003900220EA
:1015000004900520059001A90A48FFF7F7F910207B
:10151000019001A90748FFF7F1F98020019001A986
:101520000548FFF7EBF906B010BD000000300140A0
:101530003038024000040240000002402DE9FC4720
:101540000446884617461D46002001908146606883
:10155000B0F5827F0DD1A06858B9042084F85100FD
:101560003B46424641462046009500F0F8F8BDE86B
:10157000FC8700BF94F85000012801D10220F6E753
:10158000012084F8500000BFFFF7C6FA064694F821
:101590005100012802D04FF00209D6E0B8F1000F47
:1015A00000D017B94FF00109CFE0042084F85100B2
:1015B00000206065C4F83880A787E7872063A0868D
:1015C000E08620646064A06AB0F5005F10D100BFBF
:1015D0002068006820F400502168086020680068D6
:1015E00040F400502168086000BFE08F401EE08793
:1015F000A068B0F5004F0BD12068006820F04000D3
:10160000216808602068006820F480402168086034
:101610002068006800F04000402805D0206800687D
:1016200040F0400021680860E068F8B91AE02068DE
:10163000806800F0010050B12068007BA16B087049
:10164000A06B401CA063E08F401EE0870AE0FFF71C
:1016500063FA801BA84201D3681C00B915B94FF08A
:10166000030972E0E08F0028E1D11EE01AE0206853
:10167000806800F0010050B12068C068A16B08804C
:10168000A06B801CA063E08F401EE0870AE0FFF79C
:1016900043FA801BA84201D3681C00B915B94FF06A
:1016A000030952E0E08F0028E1D1A06AB0F5005FA5
:1016B00030D12068006840F48050216808602B46D3
:1016C000012211462046009600F01AFE10B14FF09C
:1016D00003093AE0E068B0F5006F04D12068C06803
:1016E000A16B088003E02068007BA16B08702B468B
:1016F000012211462046009600F002FE30B1606DD6
:1017000040F0020060654FF003091EE02068C068E9
:10171000019000BF32462946204600F070FD08B116
:10172000202060652068806800F01000102807D134
:10173000606D40F0020060654FF6EF7021688860D0
:10174000606D08B14FF0010900BF012084F851001D
:1017500000BF002084F8500000BF484607E72DE98D
:10176000F04F85B00446884691461D460E9E0020E7
:101770000490012002900020019000BF94F85000D6
:10178000012803D1022005B0BDE8F08F012084F8C4
:10179000500000BFFFF7C0F9074694F851B06068E9
:1017A0000390AA46BBF1010F0BD00398B0F5827FDE
:1017B00004D1A06810B9BBF1040F02D0022001903F
:1017C0002CE1B8F1000F03D0B9F1000F00D015B92A
:1017D0000120019022E194F85100042802D0052054
:1017E00084F8510000206065C4F83890E587A5872B
:1017F000C4F83080E586A58620646064A06AB0F5F0
:10180000005F0DD100BF2068006820F400502168FF
:1018100008602068006840F400502168086000BF3C
:101820002068006800F04000402805D0206800686B
:1018300040F0400021680860E068B0F5006F56D1C4
:10184000606810B1BAF1010F09D1206B00882168DE
:10185000C860206B801C2063E08E401EE0863FE065
:101860002068806800F0020002281CD1E08ED0B110
:101870000298012817D1206B00882168C860206B6E
:10188000801C2063E08E401EE08600200290E08EE7
:1018900048B9A06AB0F5005F05D12068006840F43F
:1018A0008050216808602068806800F0010068B1FD
:1018B000E08F58B12068C068A16B0880A06B801CC5
:1018C000A063E08F401EE08701200290FFF724F91B
:1018D000C01BB04204D3701C10B1032001909DE0E6
:1018E000E08E0028BCD1E08F0028B9D156E06068B6
:1018F00010B1BAF1010F09D1206B0078216808738B
:10190000206B401C2063E08E401EE08640E0206893
:10191000806800F0020002281CD1E08ED0B102984D
:10192000012817D1206B007821680873206B401CB8
:101930002063E08E401EE08600200290E08E48B9D1
:10194000A06AB0F5005F05D12068006840F48050BF
:10195000216808602068806800F0010068B1E08FAD
:1019600058B12068C068A16B0870A06B401CA063D0
:10197000E08F401EE08701200290FFF7CDF8C01BEA
:10198000B04201D3701C00B916B90320019045E0A4
:10199000E08E0028BBD1E08F0028B8D1A06AB0F556
:1019A000005F12D13346012211462046009700F015
:1019B000A7FC30B1606D40F002006065032001902B
:1019C0002CE02068C068049000BF2068806800F0A8
:1019D0001000102809D1606D40F0020060654FF6DC
:1019E000EF7021688860012001903A463146204618
:1019F00000F050FC20B101200190202060650DE036
:101A0000A06850B900BF002000902068C068009016
:101A100020688068009000BF00BF00BF012084F8EC
:101A2000510000BF002084F8500000BF0198AAE6D2
:101A3000042808D14FF0E021096941F004014FF07A
:101A4000E022116107E04FF0E021096921F0040173
:101A50004FF0E0221161704770B504462546681EBC
:101A6000B0F1807F01D301200FE0681E4FF0E0212C
:101A700048610F214FF0FF3001F048F800204FF08F
:101A8000E021886107200861002070BD70B5044620
:101A90000D46164600BF94F83C00012801D10220F3
:101AA00070BD012084F83C0000BF36B1042E1BD06D
:101AB000082E31D00C2E5ED145E02946206800F07A
:101AC00019FD2068806940F008002168886120685D
:101AD000806920F004002168886120688069296994
:101AE00008432168886147E02946206800F03AFDF4
:101AF0002068806940F400602168886120688069FE
:101B000020F480602168886120688069296940EA42
:101B10000120216888612FE02946206800F060FDDF
:101B20002068C06940F008002168C8612068C06969
:101B300020F004002168C8612068C0692969084351
:101B40002168C86118E02946206800F085FD2068FA
:101B5000C06940F400602168C8612068C06920F451
:101B600080602168C8612068C069296940EA012055
:101B70002168C86100E000BF00BF00BF002084F8FA
:101B80003C0000BF00BF8BE710B504460CB9012034
:101B900010BD94F83D0028B9002084F83C00204690
:101BA00000F026F8022084F83D00211D206800F096
:101BB00023FC012084F8460000BF84F83E00012188
:101BC0003F200155402001554120015500BF00BF75
:101BD000012084F84200432001554420015545204E
:101BE000015500BF012084F83D000020D0E700002F
:101BF00010B586B004462068B0F1804F34D100BFE4
:101C000000BF002000901948006840F0010017490B
:101C100008600846006800F00100009000BF00BFA7
:101C200000BF00BF00BF00200090104810300068C7
:101C300040F001000D49103108600846006800F0CE
:101C40000100009000BF00BF00BF042001900220EF
:101C5000029001200390022004900120059001A928
:101C60000348FEF74BFE00BF06B010BD30380240FF
:101C70000000024070B504460D4615B994F83E00C8
:101C80000BE0042D02D13F20005D06E0082D02D1BB
:101C90004020005D01E04120005D012801D00120CD
:101CA00070BD1DB9022084F83E000EE0042D03D162
:101CB00002213F20015508E0082D03D102214020D8
:101CC000015502E0022141200155012229462068E8
:101CD00000F0FEFB23492068884203D02249206897
:101CE000884201D1012000E0002028B12068406C2A
:101CF00040F40040216848641A49206888421BD09B
:101D00002068B0F1804F17D018492068884213D05E
:101D10001749206888420FD01649206888420BD0A6
:101D200011492068884207D013492068884203D0AF
:101D30001249206888420CD12068806800F00706AC
:101D4000062E0CD02068006840F001002168086071
:101D500005E02068006840F001002168086000206C
:101D60009EE7000000000140000401400004004024
:101D700000080040000C00400040014000180040F6
:101D80007047704701460022002391F83D2091F8EA
:101D90003E3042EA030070472DE9F84F04462068C0
:101DA00005682068C668206847694FF00009CA4680
:101DB00005F00F09B9F1000F0AD105F0200038B184
:101DC00006F0200020B1204600F0A5FCBDE8F88F09
:101DD000B9F1000F72D007F0010018B906F4907045
:101DE00000286BD005F0010030B106F4807018B106
:101DF000206C40F00100206405F0040030B107F0D1
:101E0000010018B1206C40F00200206405F00200CF
:101E100030B107F0010018B1206C40F004002064DC
:101E200005F0080048B106F0200010B907F00100E5
:101E300018B1206C40F008002064206C70B305F0ED
:101E4000200028B106F0200010B1204600F063FC0D
:101E500020684069C0F3801A206C00F0080010B9B7
:101E6000BAF1000F23D0204600F02AFC2068406918
:101E700000F04000402816D12068406920F0400062
:101E800021684861A06B50B15648A16B0865A06BF2
:101E9000FEF71FFD10B1A06B016D88470CE02046D6
:101EA000FFF76FFF08E02046FFF76BFF04E02046D6
:101EB000FFF767FF0020206488E7FFE7206B012819
:101EC00079D105F01000002875D006F01000002828
:101ED00071D000BF0020009020680068009020684A
:101EE0004068009000BF00BF2068406900F04000DB
:101EF000402839D1A06B006840681FFA80F8B8F11B
:101F0000000F30D0A08D40452DDDA4F82E80A06BB1
:101F1000C069B0F5807F1FD02068C06820F4807051
:101F20002168C8602068406920F00100216848618C
:101F30002068406920F0400021684861202084F832
:101F40003E00002020632068C06820F01000216857
:101F5000C860A06BFEF768FCA08DE28D801A81B28C
:101F60002046FFF70DFF31E7A08DE18D401A1FFAE3
:101F700080F8E08DE8B1B8F1000F1AD02068C06891
:101F800020F490702168C8602068406920F001004A
:101F900021684861202084F83E00002020632068EA
:101FA000C06820F010002168C86041462046FFF755
:101FB000E7FE0BE7FFE705F0800030B106F0800098
:101FC00018B1204600F03FFD00E705F0400030B1B9
:101FD00006F0400018B1204600F08DFBF6E600BF89
:101FE000F4E60000AD26000810B504460CB9012047
:101FF00010BDA06900B100E000BF94F83D0028B911
:10200000002084F83C00204600F028F8242084F8C2
:102010003D002068C06820F400502168C860204658
:1020200000F0D8FB2068006920F490402168086126
:102030002068406920F02A00216848612068C06853
:1020400040F400502168C86000202064202084F8FB
:102050003D0084F83E000020CAE7000010B586B0BD
:1020600004462D492068884254D100BF00BF00209B
:1020700000902A48006840F010002849086008468F
:10208000006800F01000009000BF00BF00BF00BF5C
:1020900000BF0020009021481438006840F0020082
:1020A0001E49143908600846006800F002000090DC
:1020B00000BF00BF00BF00BF00BF00200090084667
:1020C000006840F0020008600846006800F0020066
:1020D000009000BF00BF00BF40200190022002908E
:1020E00001200390022004900720059001A90C48CC
:1020F000FEF704FC802001900720059001A9084804
:10210000FEF7FCFB2520FEF758FD03221146252093
:10211000FEF763FD06B010BD0010014044380240D8
:102120000004024070B504460D46164694F83E0081
:10213000202816D105B10EB9012070BD00BF94F85A
:102140003C00012801D10220F7E7012084F83C007F
:1021500000BF0020206332462946204600F050FC94
:10216000EBE70220E9E700001D4A0168914236D101
:102170001C49098801F4004189BB1A49098801F406
:10218000804171B1184909780A2903D00021154A04
:10219000118024E01349098841F40041114A11805B
:1021A0001DE0114909780D2906D10E49098841F42D
:1021B00080410C4A118012E00B490978094A1288C3
:1021C000C2F30D02094B995406490988491C054A76
:1021D000118011460988C72901DD0021118070474F
:1021E000001001400C0000200E0000202400002000
:1021F000704700BFFEE700BFFEE770477047F8B5C5
:1022000004460E4615466068B0F5827F0DD1A06881
:10221000B0F5004F03D0A068B0F5806F05D12068FD
:10222000006820F04000216808606068B0F5827F97
:102230001FD1A068B0F5806F0DD0334600228021F9
:102240002046009500F05CF808B3606D40F0200077
:1022500060650320F8BD3346002201212046009529
:1022600000F04EF898B1606D40F0200060650320EA
:10227000F0E73346002201212046009500F040F8A7
:1022800028B1606D40F0200060650320E2E7002087
:10229000E0E700007CB504460D4616461648006887
:1022A0001821B0FBF1F01549B0FBF1F04FF47A7151
:1022B000484301906068B0F5827F0DD12B46002223
:1022C00080212046009600F01BF898B1606D40F028
:1022D0002000606503207CBD00BF019800B908E0C4
:1022E0000198401E019020688068C0F3C01000284B
:1022F000F3D100BF0020EEE70000002040420F00B5
:102300002DE9F84F04460D4690461E46DDF828900C
:10231000FEF702FCA0EB0900371AFEF7FDFB824630
:102320002C480068C0F3CB307843009045E0701C27
:10233000002842D0FEF7F0FBA0EB0A00B84200D222
:10234000A7BB2068406820F0E00021684860606812
:10235000B0F5827F0DD1A068B0F5004F03D0A06822
:10236000B0F5806F05D12068006820F0400021683A
:102370000860A06AB0F5005F0DD100BF206800685A
:1023800020F40050216808602068006840F4005084
:102390002168086000BF012084F8510000BF0020C0
:1023A00084F8500000BF0320BDE8F88FFFE70098D5
:1023B00000B900270098401E0090206880682840DF
:1023C000A84201D1012000E000204045AFD100200B
:1023D000EAE7000000000020704710B5FEF7A2FBFE
:1023E00010BD00000348006840F470000149086017
:1023F0007047000088ED00E010B50268294B984254
:102400000ED0B0F1804F0BD0274B984208D0274B0D
:10241000984205D0264B984202D0264B984203D1D1
:1024200022F070024B681A431E4B984220D0B0F144
:10243000804F1DD01C4B98421AD01C4B984217D08D
:102440001B4B984214D01B4B984211D01A4B984208
:102450000ED01A4B98420BD0194B984208D0194B0A
:10246000984205D0184B984202D0184B984203D19D
:1024700022F44072CB681A4322F080034C6943EA8D
:10248000040202608B68C3620B688362054B98424A
:1024900002D0084B984201D10B69036301234361C9
:1024A00010BD000000000140000400400008004092
:1024B000000C004000040140004001400044014085
:1024C0000048014000180040001C0040002000406F
:1024D00030B501F01F05012404FA05F3046A9C439A
:1024E0000462046A01F01F0502FA05F52C43046238
:1024F00030BD000030B5056A25F001050562026AAD
:102500004368846924F0700424F003040D682C43AC
:1025100022F002028D682A43104DA84200D103E048
:102520000F4DA84206D100BF22F00802CD682A4311
:1025300022F00402094DA84202D0094DA84207D159
:1025400023F4807323F400734D692B438D692B436F
:10255000436084614D684563026230BD0000014004
:102560000004014030B5056A25F010050562026AD5
:102570004368846924F4E04424F440740D6844EA18
:10258000052422F020028D6842EA0512124DA8426D
:1025900000D103E0114DA84207D100BF22F0800214
:1025A000CD6842EA051222F040020B4DA84202D04B
:1025B0000A4DA84209D123F4806323F400634D69D6
:1025C00043EA85038D6943EA8503436084614D686E
:1025D0008563026230BD000000000140000401403C
:1025E00030B5056A25F480750562026A4368C469DE
:1025F00024F0700424F003040D682C4322F40072CC
:102600008D6842EA0522124DA84200D103E0114D27
:10261000A84207D100BF22F40062CD6842EA052239
:1026200022F480620A4DA84202D00A4DA84209D184
:1026300023F4805323F400534D6943EA05138D6955
:1026400043EA05134360C4614D68C563026230BD4F
:10265000000001400004014030B5056A25F48055B2
:102660000562036A4468C26922F4E04222F44072BF
:102670000D6842EA052223F400538D6843EA0533CE
:10268000084DA84202D0084DA84204D124F4804449
:102690004D6944EA85144460C2614D680564036273
:1026A00030BD0000000001400004014070B5054647
:1026B000AC6B0020E085E0842046FFF762FB70BD34
:1026C0000168C96821F490710268D16001684969A4
:1026D00021F0010102685161016B012905D10168F6
:1026E000C96821F010010268D160202180F83E10F5
:1026F00000210163704710B504462068C06820F0CF
:1027000040002168C860202084F83D002046FFF783
:102710006FFD002010BD70B5044694F83E002228DD
:1027200056D1A068B0F5805F0CD1206950B9002562
:10273000A66A20684068C0F308003080A06A801C48
:10274000A06215E0A56A0026A068B0F5805F03D0FE
:10275000A06828B9206918B920684068287004E08A
:102760002068406800F07F002870A06A401CA062CA
:10277000E08D401E80B2E08540BB2068C06820F03C
:1027800020002168C8602068C06820F4807021683B
:10279000C8602068406920F001002168486120205D
:1027A00084F83E00206B01280AD12068C06820F020
:1027B00010002168C860A18D2046FFF7E1FA02E011
:1027C0002046FFF7D1FC0020206370BD0020FCE70D
:1027D0000220FAE72DE9F84F04462068006920F44A
:1027E0004050E1680843216808612169A0680843F6
:1027F00061690843E169084300902068C06849F2B4
:102800000C618843009908432168C86020684069CA
:1028100020F44070A1690843216848617649206826
:10282000884203D075492068884203D1FEF700FB37
:10283000814602E0FEF7ECFA8146E069B0F5004F10
:102840006CD102206168A0FB015003461920A9FB4E
:10285000007001462A463846FDF711FD6421B0FBA1
:10286000F1F04FEA001A02206168A0FB01510B460B
:102870001920A9FB00712A463846FDF700FD834662
:1028800002206168A0FB015003461920A9FB0071DA
:102890002A463846FDF7F3FC6421B0FBF1F000EB6B
:1028A000C00101EB0010ABEB8000322101EBC00056
:1028B0006421B0FBF1F000F0F8000AEB400A0220BE
:1028C0006168A0FB015003461920A9FB0070014676
:1028D0002A463846FDF7D3FC834602206168A0FBF8
:1028E000015003461920A9FB00712A463846FDF71E
:1028F000C6FC6421B0FBF1F000EBC00101EB00105D
:10290000ABEB8000322101EBC0006421B0FBF1F0A1
:1029100000F007005044216888606AE00420616884
:10292000A0FB015003461920A9FB007001462A466E
:102930003846FDF7A4FC824604206168A0FB0150E4
:1029400003461920A9FB007001462A463846FDF7C8
:1029500096FC6421B0FBF1F000EBC00101EB00102C
:10296000AAEB8000322101EB00106421B0FBF1F0F2
:1029700000F0F00A04206168A0FB017003461920F2
:10298000A9FB00513A462846FDF779FC6421B0FBCB
:10299000F1F00AEB001A04206168A0FB01510B461C
:1029A0001920A9FB00712A463846FDF768FC8346CA
:1029B00004206168A0FB015003461920A9FB0070A8
:1029C00001462A463846FDF75AFC6421B0FBF1F077
:1029D00000EBC00101EB0010ABEB8000322101EBFA
:1029E00000106421B0FBF1F000F00F0050442168AA
:1029F0008860BDE8F88F000000100140001401401D
:102A000010B5034699629A85DA8500201864222061
:102A100083F83E0000BF002083F83C0000BF186828
:102A2000C06840F480701C68E0601868406940F03D
:102A300001001C6860611868C06840F020001C68D4
:102A4000E060002010BD014691F83D00212828D10A
:102A50008868B0F5805F0BD1086948B90A6A1088A8
:102A6000C0F308000B685860086A801C086205E023
:102A70000B6A581C086218780B685860C88C401E96
:102A800080B2C88458B90868C06820F080000B681C
:102A9000D8600868C06840F040000B68D86000202B
:102AA00070470220FCE7000070B500240F4D10486D
:102AB000FFF772F900BF03E0641CAC4200D904E0E8
:102AC0000B48FFF75FF92028F6D100BF002403E090
:102AD000641CAC4200D906E0012206490448FFF715
:102AE00021FB0028F4D100BF70BD0000FFFF0100F2
:102AF000EC0000200E00002000BFFEE70248006846
:102B0000C0F30220704700000CED00E010B5002873
:102B100004DB0A07130E054A135406E00A07140ED5
:102B2000034A00F00F031B1FD45410BD00E400E063
:102B300018ED00E000BF704710B504460420FEF712
:102B400077FF0148046010BD0400002070B5044602
:102B50004FF4077094FBF0F594FBF0F100FB114685
:102B600003E0074800F00EF86D1E002DF9D12EB1DC
:102B70004FF47A7106FB01F000F004F870BD00001C
:102B8000603D080070B5034600224FF0E0267569ED
:102B90000D4E366803FB06F44FF0E026B16910E0F5
:102BA0004FF0E026B06988420BD0884202D20E1A5C
:102BB000324402E02E1A0E4432440146A24200D3AF
:102BC00000E0EDE700BF70BD0400002000BF054A33
:102BD000126802F04002002AF9D0C2B2014B5A60DA
:102BE000704700000010014030B587B004460D4624
:102BF0001C216846FDF736FC4FF080400E49086006
:102C00000846456000218160C460FEF7BDFF60207A
:102C10000090204604EBD0714910019102200290EF
:102C2000082269460448FEF731FF08210248FFF7F1
:102C300021F807B030BD0000FC020020FDF77EFF48
:102C40000723022208214FF4A87000F059F8A820A9
:102C5000FFF772FF4FF4E13000F0C0F814210320B9
:102C6000FFF7C2FFFDF7E2FC00F00EF802A0FDF74F
:102C70007DFB00BFFEE7000048656C6C6F20576F5E
:102C8000726C64210D0A000008B500BF00BF00206F
:102C900000901848006840F48050164908600846C3
:102CA000006800F48050009000BF00BF00BF1248D1
:102CB000124908604FF48270486000210F4881601B
:102CC000C160016141614FF4007181613021C161D6
:102CD00000210162416281620721C162FEF75EFB51
:102CE00006480068006840F0400004490968086030
:102CF00008BD000044380240003001405C02002062
:102D00002DE9F04192B080460C4615461E4600273C
:102D1000302106A8FDF7A6FB142101A8FDF7A2FBB0
:102D200000BF002000902A48006840F080502849E9
:102D300008600846006800F08050009000BF00BFA7
:102D400000BF002000902348006840F480402149E3
:102D500008600846006800F48040009000BF00BF93
:102D6000012006900004079002200C9041050D916F
:102D7000CDF83C800E941095119606A8FEF7C0F889
:102D800007461FB1012012B0BDE8F0810F2001906D
:102D900002200290002003904FF4A05004904FF4C2
:102DA00080500590052101A8FDF76AFF07460FB185
:102DB0000120E8E7FDF7AAFE41F20101884205D1B2
:102DC0000548006840F48070034908600020DAE795
:102DD0004038024000700040003C024010B50446FC
:102DE00009480A4908600846446000218160C160C2
:102DF000016181610C214161FFF7F6F8012204496C
:102E00000248FFF78FF910BD00100140EC000020D0
:102E10000E0000204FF04070E1EE100A70470000F5
:102E2000000000000000010203040607080900007A
:102E30000000010203040000582E000800000020DA
:102E400024000000C40100087C2E0008240000209B
:102E500084070000E00100080024F40000000000E6
:102E60000000000000000000000000001000000052
:0C2E700001000000000000000000000055
:040000050800018965
:00000001FF
